:1000000002C01895E1C08FE181BD87E181BD8FED10
:100010008DBFC0EDE1EB4E2EDD275D2E662487EE11
:1000200087BBC198C298C0987894002786B384FB98
:100030000EF401E041E0041709F002C06EC001C0F7
:1000400000C0C09AC19886E960D1C19ACAD0A0E622
:10005000B0E02C93A1E6B0E01C934FEFA0E6B0E037
:100060000C91041709F001C0ECCFA1E6B0E00C91AF
:100070004FEB0423A1E6B0E00C93A0E6B0E08C9136
:10008000A4E6B0E08C93A1E6B0E08C91A3E6B0E0EA
:100090008C93E1E0F0E025D1C198E1E0F0E021D1DE
:1000A000E1E0F0E0A4E6B0E091E005D1E2E0F0E0CC
:1000B000A3E6B0E091E0FFD000C0C29886E925D168
:1000C000C29A8FD0A0E6B0E02C93A1E6B0E01C93DA
:1000D0004FEFA0E6B0E00C91041709F001C0EDCF9E
:1000E000A1E6B0E00C914FEB0423A1E6B0E00C9345
:1000F000A1E6B0E08C91A2E6B0E08C93E1E0F0E004
:10010000F0D0C298E2E0F0E0ECD0E3E0F0E0A2E66C
:10011000B0E091E0D0D0C09800C0E1E0F0E0A4E60B
:10012000B0E091E0D3D04FEFA4E6B0E00C9104171B
:1001300009F001C086CFE1E0F0E0A4E6B0E091E094
:10014000C5D0E2E0F0E0A3E6B0E091E0BFD0E3E0AC
:10015000F0E0A2E6B0E091E0B9D043D0A0E6B0E094
:100160002C93A1E6B0E01C93A1E6B0E00C914FEB1C
:100170000423A1E6B0E00C93C198C298A4E6B0E0D5
:100180004C91A0E6B0E00C91041709F01AC0A3E668
:10019000B0E04C91A1E6B0E00C91041709F003C067
:1001A000C298C19A0EC0A2E6B0E04C91A1E6B0E0C0
:1001B0000C91041709F003C0C29AC19802C0C198FB
:1001C000C298CBCFF894FFCF8F939F938FB733957F
:1001D000539509F443959FE392BF9F918FBF8F91F1
:1001E00018950F933F934F935F932F923F928F9366
:1001F0009F938FB78F9383B78F93816083BF89B7A6
:100200008F93826089BF8FE382BF552744273327AE
:10021000483008F03FC037331CF4B39BF8CFF8CF19
:100220004830C4F5B399FCCF332731319CF5B39BEB
:10023000FCCF932F3327292E2694322C290E990F89
:10024000390E32153CF5B399FCCF33270CE011275A
:1002500022273215F0F3B39909C08894111F221F89
:100260003315C4F4B39BFCCF332708C00894111F87
:10027000221F33157CF4B399FCCF33270A9549F735
:10028000912F991F221F991F221F25FB16F91F77F7
:100290002F7102C01FEF2FEF8F9189BF8F9183BF06
:1002A0008F918FBF9F918F913F902F905F914F9132
:1002B0003F910F910895E199FECFEEBB8D918DBBDB
:1002C000E29AE19A31969A95B1F70895E199FECFB5
:1002D000EEBBE09AE09A8DB38D9331969A95B1F783
:1002E000089524E08AEF11D02A95E1F73197882705
:1002F0008E2B8F2BB1F708950A95F1F70895689426
:1003000062F80895E89462F8089531E099279A9583
:0E0310000000E9F73A95D9F78A95B9F70895F4
:00000001FF
